 sspi_bridge

 Timestamp is ffffffff (Sun Feb  7 06:28:15 2106)

 Preferred load address is 10000000

 Start         Length     Name                   Class
 0001:00000000 00000020H .text$di                CODE
 0001:00000020 00003ab0H .text$mn                CODE
 0001:00003ad0 0000001dH .text$x                 CODE
 0002:00000000 00000120H .idata$5                DATA
 0002:00000120 00000004H .00cfg                  DATA
 0002:00000124 00000004H .CRT$XCA                DATA
 0002:00000128 00000004H .CRT$XCU                DATA
 0002:0000012c 00000004H .CRT$XCZ                DATA
 0002:00000130 00000004H .CRT$XIA                DATA
 0002:00000134 00000004H .CRT$XIZ                DATA
 0002:00000138 00000004H .CRT$XPA                DATA
 0002:0000013c 00000004H .CRT$XPZ                DATA
 0002:00000140 00000004H .CRT$XTA                DATA
 0002:00000144 00000004H .CRT$XTZ                DATA
 0002:00000148 00000000H .gfids$y                DATA
 0002:00000148 00000e20H .rdata                  DATA
 0002:00000f68 0000012cH .rdata$r                DATA
 0002:00001094 00000008H .rdata$sxdata           DATA
 0002:0000109c 000002e4H .rdata$zzzdbg           DATA
 0002:00001380 00000004H .rtc$IAA                DATA
 0002:00001384 00000004H .rtc$IZZ                DATA
 0002:00001388 00000004H .rtc$TAA                DATA
 0002:0000138c 00000004H .rtc$TZZ                DATA
 0002:00001390 00000170H .xdata$x                DATA
 0002:00001500 00000360H .edata                  DATA
 0002:00001860 000000a0H .idata$2                DATA
 0002:00001900 00000014H .idata$3                DATA
 0002:00001914 00000120H .idata$4                DATA
 0002:00001a34 000005e0H .idata$6                DATA
 0003:00000000 00000048H .data                   DATA
 0003:00000048 00000078H .data$r                 DATA
 0003:000000c0 00000374H .bss                    DATA
 0004:00000000 00000060H .rsrc$01                DATA
 0004:00000060 00000330H .rsrc$02                DATA

  Address         Publics by Value              Rva+Base       Lib:Object

 0000:00000000       ___guard_iat_count         00000000     <absolute>
 0000:00000000       ___arm64x_redirection_metadata 00000000     <absolute>
 0000:00000000       ___hybrid_code_map_count   00000000     <absolute>
 0000:00000000       ___guard_iat_table         00000000     <absolute>
 0000:00000000       ___hybrid_code_map         00000000     <absolute>
 0000:00000000       ___arm64x_redirection_metadata_count 00000000     <absolute>
 0000:00000000       ___guard_eh_cont_count     00000000     <absolute>
 0000:00000000       ___arm64x_extra_rfe_table_size 00000000     <absolute>
 0000:00000000       ___hybrid_auxiliary_iat    00000000     <absolute>
 0000:00000000       ___guard_fids_table        00000000     <absolute>
 0000:00000000       ___guard_longjmp_count     00000000     <absolute>
 0000:00000000       ___volatile_metadata       00000000     <absolute>
 0000:00000000       ___enclave_config          00000000     <absolute>
 0000:00000000       ___arm64x_native_entrypoint 00000000     <absolute>
 0000:00000000       ___dynamic_value_reloc_table 00000000     <absolute>
 0000:00000000       ___guard_longjmp_table     00000000     <absolute>
 0000:00000000       ___arm64x_extra_rfe_table  00000000     <absolute>
 0000:00000000       ___x64_code_ranges_to_entry_points 00000000     <absolute>
 0000:00000000       ___guard_eh_cont_table     00000000     <absolute>
 0000:00000000       ___AbsoluteZero            00000000     <absolute>
 0000:00000000       ___guard_fids_count        00000000     <absolute>
 0000:00000000       ___x64_code_ranges_to_entry_points_count 00000000     <absolute>
 0000:00000002       ___safe_se_handler_count   00000002     <absolute>
 0000:00000100       ___guard_flags             00000100     <absolute>
 0000:00000000       ___ImageBase               10000000     <linker-defined>
 0001:00000020       ?StringCchCopyW@@YGJPAGIPBG@Z 10001020 f i sspi.obj
 0001:0000008e       ___local_stdio_printf_options 1000108e f i sspi.obj
 0001:00000094       __vfprintf_l               10001094 f i sspi.obj
 0001:000000b8       __vsprintf_s_l             100010b8 f i sspi.obj
 0001:000000e7       _dump                      100010e7 f   sspi.obj
 0001:00000200       _fprintf                   10001200 f i sspi.obj
 0001:00000306       _gss_accept_sec_context    10001306 f   sspi.obj
 0001:0000037b       _gss_acquire_cred          1000137b f   sspi.obj
 0001:00000781       _gss_add_oid_set_member    10001781 f   sspi.obj
 0001:000008b0       _gss_canonicalize_name     100018b0 f   sspi.obj
 0001:000009b1       _gss_compare_name          100019b1 f   sspi.obj
 0001:00000b13       _gss_context_time          10001b13 f   sspi.obj
 0001:00000bd6       _gss_create_empty_oid_set  10001bd6 f   sspi.obj
 0001:00000c44       _gss_delete_sec_context    10001c44 f   sspi.obj
 0001:00000ce9       _gss_display_name          10001ce9 f   sspi.obj
 0001:00000df6       _gss_display_status        10001df6 f   sspi.obj
 0001:00000ee9       _gss_export_name           10001ee9 f   sspi.obj
 0001:00001052       _gss_export_sec_context    10002052 f   sspi.obj
 0001:0000108c       _gss_get_mic               1000208c f   sspi.obj
 0001:00001195       _gss_import_name           10002195 f   sspi.obj
 0001:0000140d       _gss_import_sec_context    1000240d f   sspi.obj
 0001:0000144e       _gss_indicate_mechs        1000244e f   sspi.obj
 0001:0000156c       _gss_init_sec_context      1000256c f   sspi.obj
 0001:00001acb       _gss_inquire_context       10002acb f   sspi.obj
 0001:00001d5d       _gss_inquire_cred          10002d5d f   sspi.obj
 0001:00001ea0       _gss_inquire_names_for_mech 10002ea0 f   sspi.obj
 0001:00001f61       _gss_release_buffer        10002f61 f   sspi.obj
 0001:00001fb6       _gss_release_cred          10002fb6 f   sspi.obj
 0001:00002042       _gss_release_name          10003042 f   sspi.obj
 0001:000020a7       _gss_release_oid_set       100030a7 f   sspi.obj
 0001:00002121       _gss_unwrap                10003121 f   sspi.obj
 0001:000022bb       _gss_verify_mic            100032bb f   sspi.obj
 0001:000023ac       _gss_wrap                  100033ac f   sspi.obj
 0001:000025b7       _gss_wrap_size_limit       100035b7 f   sspi.obj
 0001:000029f3       _sprintf_s                 100039f3 f i sspi.obj
 0001:00002a0f       _FreeContextBuffer@4       10003a0f f   secur32:Secur32.dll
 0001:00002a15       _EncryptMessage@16         10003a15 f   secur32:Secur32.dll
 0001:00002a1b       _DecryptMessage@16         10003a1b f   secur32:Secur32.dll
 0001:00002a21       ??3@YAXPAXI@Z              10003a21 f   MSVCRT:delete_scalar_size.obj
 0001:00002a2f       ??_V@YAXPAX@Z              10003a2f f   MSVCRT:delete_array.obj
 0001:00002a34       ___raise_securityfailure   10003a34 f   MSVCRT:gs_report.obj
 0001:00002a5c       ___report_gsfailure        10003a5c f   MSVCRT:gs_report.obj
 0001:00002b55       ___report_rangecheckfailure 10003b55 f   MSVCRT:gs_report.obj
 0001:00002b61       ___report_securityfailure  10003b61 f   MSVCRT:gs_report.obj
 0001:00002c2f       ??2@YAPAXIABUnothrow_t@std@@@Z 10003c2f f   MSVCRT:new_scalar_nothrow.obj
 0001:00002c84       ??_U@YAPAXIABUnothrow_t@std@@@Z 10003c84 f   MSVCRT:new_array_nothrow.obj
 0001:00002c8d       @__security_check_cookie@4 10003c8d f   MSVCRT:secchk.obj
 0001:00002ca0       __alldiv                   10003ca0 f   MSVCRT:lldiv.obj
 0001:0000308a       __DllMainCRTStartup@12     1000408a f   MSVCRT:dll_dllmain.obj
 0001:000030ad       ??3@YAXPAX@Z               100040ad f   MSVCRT:delete_scalar.obj
 0001:000030b2       ??2@YAPAXI@Z               100040b2 f   MSVCRT:new_scalar.obj
 0001:0000312f       ___security_init_cookie    1000412f f   MSVCRT:gs_support.obj
 0001:0000317a       _DllMain@12                1000417a f   MSVCRT:dll_dllmain_stub.obj
 0001:0000319c       ?__scrt_initialize_type_info@@YAXXZ 1000419c f   MSVCRT:tncleanup.obj
 0001:000031a8       ?__scrt_uninitialize_type_info@@YAXXZ 100041a8 f   MSVCRT:tncleanup.obj
 0001:000031b4       ___local_stdio_scanf_options 100041b4 f i MSVCRT:default_local_stdio_options.obj
 0001:000031ba       ___scrt_initialize_default_local_stdio_options 100041ba f   MSVCRT:default_local_stdio_options.obj
 0001:0000321b       ___scrt_acquire_startup_lock 1000421b f   MSVCRT:utility.obj
 0001:0000324d       ___scrt_dllmain_after_initialize_c 1000424d f   MSVCRT:utility.obj
 0001:00003278       ___scrt_dllmain_before_initialize_c 10004278 f   MSVCRT:utility.obj
 0001:00003286       ___scrt_dllmain_crt_thread_attach 10004286 f   MSVCRT:utility.obj
 0001:000032a5       ___scrt_dllmain_crt_thread_detach 100042a5 f   MSVCRT:utility.obj
 0001:000032b2       ___scrt_dllmain_exception_filter 100042b2 f   MSVCRT:utility.obj
 0001:000032e6       ___scrt_dllmain_uninitialize_c 100042e6 f   MSVCRT:utility.obj
 0001:00003309       ___scrt_dllmain_uninitialize_critical 10004309 f   MSVCRT:utility.obj
 0001:00003316       ___scrt_initialize_crt     10004316 f   MSVCRT:utility.obj
 0001:0000334f       ___scrt_initialize_onexit_tables 1000434f f   MSVCRT:utility.obj
 0001:000033d6       ___scrt_is_nonwritable_in_current_image 100043d6 f   MSVCRT:utility.obj
 0001:0000346a       ___scrt_release_startup_lock 1000446a f   MSVCRT:utility.obj
 0001:00003487       ___scrt_uninitialize_crt   10004487 f   MSVCRT:utility.obj
 0001:000034af       ___scrt_get_dyn_tls_init_callback 100044af f   MSVCRT:dyn_tls_init.obj
 0001:000034b5       ___scrt_fastfail           100044b5 f   MSVCRT:utility_desktop.obj
 0001:000035cf       __crt_debugger_hook        100045cf f   MSVCRT:utility_desktop.obj
 0001:000035d7       __RTC_Initialize           100045d7 f   MSVCRT:initsect.obj
 0001:00003603       __RTC_Terminate            10004603 f   MSVCRT:initsect.obj
 0001:00003630       __SEH_prolog4              10004630 f   MSVCRT:sehprolg4.obj
 0001:00003674       __SEH_epilog4              10004674 f   MSVCRT:sehprolg4.obj
 0001:00003688       __except_handler4          10004688 f   MSVCRT:chandler4gs.obj
 0001:000036b7       @_guard_check_icall_nop@4  100046b7 f i MSVCRT:guard_support.obj
 0001:000036ba       ??0bad_alloc@std@@QAE@ABV01@@Z 100046ba f i MSVCRT:throw_bad_alloc.obj
 0001:000036d5       ??0bad_alloc@std@@QAE@XZ   100046d5 f i MSVCRT:throw_bad_alloc.obj
 0001:000036ed       ??0bad_array_new_length@std@@QAE@ABV01@@Z 100046ed f i MSVCRT:throw_bad_alloc.obj
 0001:00003708       ??0bad_array_new_length@std@@QAE@XZ 10004708 f i MSVCRT:throw_bad_alloc.obj
 0001:00003720       ??0exception@std@@QAE@ABV01@@Z 10004720 f i MSVCRT:throw_bad_alloc.obj
 0001:0000374c       ??1bad_array_new_length@std@@UAE@XZ 1000474c f i MSVCRT:throw_bad_alloc.obj
 0001:0000374c       ??1bad_alloc@std@@UAE@XZ   1000474c f i MSVCRT:throw_bad_alloc.obj
 0001:0000375d       ??_Gbad_alloc@std@@UAEPAXI@Z 1000475d f i MSVCRT:throw_bad_alloc.obj
 0001:0000375d       ??_Gbad_array_new_length@std@@UAEPAXI@Z 1000475d f i MSVCRT:throw_bad_alloc.obj
 0001:0000375d       ??_Gexception@std@@UAEPAXI@Z 1000475d f i MSVCRT:throw_bad_alloc.obj
 0001:0000375d       ??_Ebad_alloc@std@@UAEPAXI@Z 1000475d f i MSVCRT:throw_bad_alloc.obj
 0001:0000375d       ??_Ebad_array_new_length@std@@UAEPAXI@Z 1000475d f i MSVCRT:throw_bad_alloc.obj
 0001:0000375d       ??_Eexception@std@@UAEPAXI@Z 1000475d f i MSVCRT:throw_bad_alloc.obj
 0001:0000378a       ?__scrt_throw_std_bad_alloc@@YAXXZ 1000478a f   MSVCRT:throw_bad_alloc.obj
 0001:000037a7       ?__scrt_throw_std_bad_array_new_length@@YAXXZ 100047a7 f   MSVCRT:throw_bad_alloc.obj
 0001:000037c4       ?what@exception@std@@UBEPBDXZ 100047c4 f i MSVCRT:throw_bad_alloc.obj
 0001:000037d1       ___isa_available_init      100047d1 f   MSVCRT:cpu_disp.obj
 0001:000039a1       __get_startup_argv_mode    100049a1 f   MSVCRT:argv_mode.obj
 0001:000039a5       ___scrt_is_ucrt_dll_in_use 100049a5 f   MSVCRT:ucrt_detection.obj
 0001:000039b1       ??_Gtype_info@@UAEPAXI@Z   100049b1 f i MSVCRT:std_type_info_static.obj
 0001:000039b1       ??_Etype_info@@UAEPAXI@Z   100049b1 f i MSVCRT:std_type_info_static.obj
 0001:000039d4       _IsProcessorFeaturePresent@4 100049d4 f   kernel32:KERNEL32.dll
 0001:000039da       _memcmp                    100049da f   vcruntime:VCRUNTIME140.dll
 0001:000039e0       _memcpy                    100049e0 f   vcruntime:VCRUNTIME140.dll
 0001:000039e6       _memset                    100049e6 f   vcruntime:VCRUNTIME140.dll
 0001:000039ec       ___CxxFrameHandler3        100049ec f   vcruntime:VCRUNTIME140.dll
 0001:000039f2       ___std_type_info_destroy_list 100049f2 f   vcruntime:VCRUNTIME140.dll
 0001:000039f8       __except_handler4_common   100049f8 f   vcruntime:VCRUNTIME140.dll
 0001:000039fe       ___std_exception_copy      100049fe f   vcruntime:VCRUNTIME140.dll
 0001:00003a04       ___std_exception_destroy   10004a04 f   vcruntime:VCRUNTIME140.dll
 0001:00003a0a       __CxxThrowException@8      10004a0a f   vcruntime:VCRUNTIME140.dll
 0001:00003a10       _free                      10004a10 f   ucrt:api-ms-win-crt-heap-l1-1-0.dll
 0001:00003a16       _malloc                    10004a16 f   ucrt:api-ms-win-crt-heap-l1-1-0.dll
 0001:00003a1c       __initterm                 10004a1c f   ucrt:api-ms-win-crt-runtime-l1-1-0.dll
 0001:00003a22       __initterm_e               10004a22 f   ucrt:api-ms-win-crt-runtime-l1-1-0.dll
 0001:00003a28       __callnewh                 10004a28 f   ucrt:api-ms-win-crt-heap-l1-1-0.dll
 0001:00003a2e       __seh_filter_dll           10004a2e f   ucrt:api-ms-win-crt-runtime-l1-1-0.dll
 0001:00003a34       __configure_narrow_argv    10004a34 f   ucrt:api-ms-win-crt-runtime-l1-1-0.dll
 0001:00003a3a       __initialize_narrow_environment 10004a3a f   ucrt:api-ms-win-crt-runtime-l1-1-0.dll
 0001:00003a40       __initialize_onexit_table  10004a40 f   ucrt:api-ms-win-crt-runtime-l1-1-0.dll
 0001:00003a46       __execute_onexit_table     10004a46 f   ucrt:api-ms-win-crt-runtime-l1-1-0.dll
 0001:00003a4c       __cexit                    10004a4c f   ucrt:api-ms-win-crt-runtime-l1-1-0.dll
 0001:00003a52       ___vcrt_thread_detach      10004a52 f   MSVCRT:ucrt_stubs.obj
 0001:00003a52       ___vcrt_thread_attach      10004a52 f   MSVCRT:ucrt_stubs.obj
 0001:00003a52       ___acrt_thread_attach      10004a52 f   MSVCRT:ucrt_stubs.obj
 0001:00003a52       ___scrt_stub_for_acrt_uninitialize 10004a52 f   MSVCRT:ucrt_stubs.obj
 0001:00003a52       ___scrt_stub_for_acrt_thread_attach 10004a52 f   MSVCRT:ucrt_stubs.obj
 0001:00003a52       ___acrt_thread_detach      10004a52 f   MSVCRT:ucrt_stubs.obj
 0001:00003a52       ___scrt_stub_for_acrt_thread_detach 10004a52 f   MSVCRT:ucrt_stubs.obj
 0001:00003a52       ___vcrt_uninitialize_critical 10004a52 f   MSVCRT:ucrt_stubs.obj
 0001:00003a52       ___vcrt_uninitialize       10004a52 f   MSVCRT:ucrt_stubs.obj
 0001:00003a52       ___vcrt_initialize         10004a52 f   MSVCRT:ucrt_stubs.obj
 0001:00003a52       ___scrt_stub_for_acrt_uninitialize_critical 10004a52 f   MSVCRT:ucrt_stubs.obj
 0001:00003a52       ___scrt_stub_for_acrt_initialize 10004a52 f   MSVCRT:ucrt_stubs.obj
 0001:00003a52       ___acrt_uninitialize       10004a52 f   MSVCRT:ucrt_stubs.obj
 0001:00003a52       ___acrt_initialize         10004a52 f   MSVCRT:ucrt_stubs.obj
 0001:00003a52       ___acrt_uninitialize_critical 10004a52 f   MSVCRT:ucrt_stubs.obj
 0001:00003a55       ___scrt_stub_for_is_c_termination_complete 10004a55 f   MSVCRT:ucrt_stubs.obj
 0001:00003a55       __is_c_termination_complete 10004a55 f   MSVCRT:ucrt_stubs.obj
 0001:00003a58       __filter_x86_sse2_floating_point_exception 10004a58 f   MSVCRT:x86_exception_filter.obj
 0001:00003a58       __filter_x86_sse2_floating_point_exception_default 10004a58 f   MSVCRT:x86_exception_filter.obj
 0002:00000000       __imp__FileTimeToSystemTime@8 10005000     kernel32:KERNEL32.dll
 0002:00000004       __imp__IsDebuggerPresent@0 10005004     kernel32:KERNEL32.dll
 0002:00000008       __imp__InitializeSListHead@4 10005008     kernel32:KERNEL32.dll
 0002:0000000c       __imp__DisableThreadLibraryCalls@4 1000500c     kernel32:KERNEL32.dll
 0002:00000010       __imp__GetCurrentThreadId@0 10005010     kernel32:KERNEL32.dll
 0002:00000014       __imp__GetCurrentProcessId@0 10005014     kernel32:KERNEL32.dll
 0002:00000018       __imp__QueryPerformanceCounter@4 10005018     kernel32:KERNEL32.dll
 0002:0000001c       __imp__IsProcessorFeaturePresent@4 1000501c     kernel32:KERNEL32.dll
 0002:00000020       __imp__TerminateProcess@8  10005020     kernel32:KERNEL32.dll
 0002:00000024       __imp__GetCurrentProcess@0 10005024     kernel32:KERNEL32.dll
 0002:00000028       __imp__SetUnhandledExceptionFilter@4 10005028     kernel32:KERNEL32.dll
 0002:0000002c       __imp__FileTimeToLocalFileTime@8 1000502c     kernel32:KERNEL32.dll
 0002:00000030       __imp__GetSystemTimeAsFileTime@4 10005030     kernel32:KERNEL32.dll
 0002:00000034       __imp__FormatMessageW@28   10005034     kernel32:KERNEL32.dll
 0002:00000038       __imp__lstrlenW@4          10005038     kernel32:KERNEL32.dll
 0002:0000003c       __imp__WideCharToMultiByte@32 1000503c     kernel32:KERNEL32.dll
 0002:00000040       __imp__CompareStringEx@36  10005040     kernel32:KERNEL32.dll
 0002:00000044       __imp__MultiByteToWideChar@24 10005044     kernel32:KERNEL32.dll
 0002:00000048       __imp__UnhandledExceptionFilter@4 10005048     kernel32:KERNEL32.dll
 0002:0000004c       \177KERNEL32_NULL_THUNK_DATA 1000504c     kernel32:KERNEL32.dll
 0002:00000050       __imp__FreeContextBuffer@4 10005050     secur32:Secur32.dll
 0002:00000054       __imp__EnumerateSecurityPackagesW@8 10005054     secur32:Secur32.dll
 0002:00000058       __imp__DecryptMessage@16   10005058     secur32:Secur32.dll
 0002:0000005c       __imp__EncryptMessage@16   1000505c     secur32:Secur32.dll
 0002:00000060       __imp__VerifySignature@16  10005060     secur32:Secur32.dll
 0002:00000064       __imp__MakeSignature@16    10005064     secur32:Secur32.dll
 0002:00000068       __imp__AcquireCredentialsHandleW@36 10005068     secur32:Secur32.dll
 0002:0000006c       __imp__QueryCredentialsAttributesW@12 1000506c     secur32:Secur32.dll
 0002:00000070       __imp__QueryContextAttributesW@12 10005070     secur32:Secur32.dll
 0002:00000074       __imp__DeleteSecurityContext@4 10005074     secur32:Secur32.dll
 0002:00000078       __imp__InitializeSecurityContextW@48 10005078     secur32:Secur32.dll
 0002:0000007c       __imp__FreeCredentialsHandle@4 1000507c     secur32:Secur32.dll
 0002:00000080       \177Secur32_NULL_THUNK_DATA 10005080     secur32:Secur32.dll
 0002:00000084       __imp__memcmp              10005084     vcruntime:VCRUNTIME140.dll
 0002:00000088       __imp__memcpy              10005088     vcruntime:VCRUNTIME140.dll
 0002:0000008c       __imp__memset              1000508c     vcruntime:VCRUNTIME140.dll
 0002:00000090       __imp____CxxFrameHandler3  10005090     vcruntime:VCRUNTIME140.dll
 0002:00000094       __imp____std_type_info_destroy_list 10005094     vcruntime:VCRUNTIME140.dll
 0002:00000098       __imp___except_handler4_common 10005098     vcruntime:VCRUNTIME140.dll
 0002:0000009c       __imp____std_exception_copy 1000509c     vcruntime:VCRUNTIME140.dll
 0002:000000a0       __imp____std_exception_destroy 100050a0     vcruntime:VCRUNTIME140.dll
 0002:000000a4       __imp___CxxThrowException@8 100050a4     vcruntime:VCRUNTIME140.dll
 0002:000000a8       \177VCRUNTIME140_NULL_THUNK_DATA 100050a8     vcruntime:VCRUNTIME140.dll
 0002:000000ac       __imp___wgetenv            100050ac     ucrt:api-ms-win-crt-environment-l1-1-0.dll
 0002:000000b0       __imp__getenv              100050b0     ucrt:api-ms-win-crt-environment-l1-1-0.dll
 0002:000000b4       \177api-ms-win-crt-environment-l1-1-0_NULL_THUNK_DATA 100050b4     ucrt:api-ms-win-crt-environment-l1-1-0.dll
 0002:000000b8       __imp__malloc              100050b8     ucrt:api-ms-win-crt-heap-l1-1-0.dll
 0002:000000bc       __imp__free                100050bc     ucrt:api-ms-win-crt-heap-l1-1-0.dll
 0002:000000c0       __imp___callnewh           100050c0     ucrt:api-ms-win-crt-heap-l1-1-0.dll
 0002:000000c4       \177api-ms-win-crt-heap-l1-1-0_NULL_THUNK_DATA 100050c4     ucrt:api-ms-win-crt-heap-l1-1-0.dll
 0002:000000c8       __imp___errno              100050c8     ucrt:api-ms-win-crt-runtime-l1-1-0.dll
 0002:000000cc       __imp___invalid_parameter_noinfo 100050cc     ucrt:api-ms-win-crt-runtime-l1-1-0.dll
 0002:000000d0       __imp___execute_onexit_table 100050d0     ucrt:api-ms-win-crt-runtime-l1-1-0.dll
 0002:000000d4       __imp___initialize_onexit_table 100050d4     ucrt:api-ms-win-crt-runtime-l1-1-0.dll
 0002:000000d8       __imp___initterm           100050d8     ucrt:api-ms-win-crt-runtime-l1-1-0.dll
 0002:000000dc       __imp___initterm_e         100050dc     ucrt:api-ms-win-crt-runtime-l1-1-0.dll
 0002:000000e0       __imp___cexit              100050e0     ucrt:api-ms-win-crt-runtime-l1-1-0.dll
 0002:000000e4       __imp___seh_filter_dll     100050e4     ucrt:api-ms-win-crt-runtime-l1-1-0.dll
 0002:000000e8       __imp___configure_narrow_argv 100050e8     ucrt:api-ms-win-crt-runtime-l1-1-0.dll
 0002:000000ec       __imp___initialize_narrow_environment 100050ec     ucrt:api-ms-win-crt-runtime-l1-1-0.dll
 0002:000000f0       \177api-ms-win-crt-runtime-l1-1-0_NULL_THUNK_DATA 100050f0     ucrt:api-ms-win-crt-runtime-l1-1-0.dll
 0002:000000f4       __imp__fflush              100050f4     ucrt:api-ms-win-crt-stdio-l1-1-0.dll
 0002:000000f8       __imp____acrt_iob_func     100050f8     ucrt:api-ms-win-crt-stdio-l1-1-0.dll
 0002:000000fc       __imp____stdio_common_vfprintf 100050fc     ucrt:api-ms-win-crt-stdio-l1-1-0.dll
 0002:00000100       __imp____stdio_common_vsprintf_s 10005100     ucrt:api-ms-win-crt-stdio-l1-1-0.dll
 0002:00000104       \177api-ms-win-crt-stdio-l1-1-0_NULL_THUNK_DATA 10005104     ucrt:api-ms-win-crt-stdio-l1-1-0.dll
 0002:00000108       __imp__wcslen              10005108     ucrt:api-ms-win-crt-string-l1-1-0.dll
 0002:0000010c       __imp___wcsdup             1000510c     ucrt:api-ms-win-crt-string-l1-1-0.dll
 0002:00000110       __imp__wcscpy_s            10005110     ucrt:api-ms-win-crt-string-l1-1-0.dll
 0002:00000114       __imp__wcscat_s            10005114     ucrt:api-ms-win-crt-string-l1-1-0.dll
 0002:00000118       __imp__wcscmp              10005118     ucrt:api-ms-win-crt-string-l1-1-0.dll
 0002:0000011c       \177api-ms-win-crt-string-l1-1-0_NULL_THUNK_DATA 1000511c     ucrt:api-ms-win-crt-string-l1-1-0.dll
 0002:00000120       ___guard_check_icall_fptr  10005120     MSVCRT:guard_support.obj
 0002:00000124       ___xc_a                    10005124     MSVCRT:initializers.obj
 0002:0000012c       ___xc_z                    1000512c     MSVCRT:initializers.obj
 0002:00000130       ___xi_a                    10005130     MSVCRT:initializers.obj
 0002:00000134       ___xi_z                    10005134     MSVCRT:initializers.obj
 0002:00000138       ___xp_a                    10005138     MSVCRT:initializers.obj
 0002:0000013c       ___xp_z                    1000513c     MSVCRT:initializers.obj
 0002:00000140       ___xt_a                    10005140     MSVCRT:initializers.obj
 0002:00000144       ___xt_z                    10005144     MSVCRT:initializers.obj
 0002:00000148       ??_C@_0BC@MKOOIHKJ@SSPI_BRIDGE_TRACE@ 10005148     sspi.obj
 0002:0000015c       ??_C@_09NLECEHAP@?$CK?$IGH?$IG?w?$BC?$AB?$AC?$AC@ 1000515c     sspi.obj
 0002:00000168       ??_C@_06EHDDNHBB@?$CL?$AG?$AB?$AF?$AF?$AC@ 10005168     sspi.obj
 0002:00000170       ??_C@_0L@ILDJNAMO@?$CK?$IGH?$IG?w?$BC?$AB?$AC?$AB?$AB@ 10005170     sspi.obj
 0002:0000017c       ??_C@_0L@IJHPGOJH@?$CK?$IGH?$IG?w?$BC?$AB?$AC?$AC?$AB@ 1000517c     sspi.obj
 0002:00000188       ??_C@_0L@PGEOCEIL@?$CK?$IGH?$IG?w?$BC?$AB?$AC?$AB?$AE@ 10005188     sspi.obj
 0002:00000194       ??_C@_06BDCPMOMO@?$CL?$AG?$AB?$AF?$AG?$AE@ 10005194     sspi.obj
 0002:0000019c       ??_C@_11LOCGONAA@@         1000519c     sspi.obj
 0002:000001a0       ??_C@_0O@EEFELDNF@?$DN?$DN?$DN?$DN?5?$CFs?5?$DN?$DN?$DN?$DN?6@ 100051a0     sspi.obj
 0002:000001b0       ??_C@_01EEMJAFIK@?6@       100051b0     sspi.obj
 0002:000001b4       ??_C@_05BFHEBJNP@?$CF02X?5@ 100051b4     sspi.obj
 0002:000001bc       ??_C@_0CN@OHCGCLJG@?$FLSSPI?3?$CFld?$FN?5?$CFs?3?5?$CF02d?1?$CF02d?1?$CFd?5?5?$CF0@ 100051bc     sspi.obj
 0002:000001ec       ??_C@_0BK@OFONCMJB@?$FLSSPI?3?$CFld?$FN?5Kerberos?5mech?6@ 100051ec     sspi.obj
 0002:00000208       ??_C@_0BI@BBDDHMFG@?$FLSSPI?3?$CFld?$FN?5SPNEGO?5mech?6@ 10005208     sspi.obj
 0002:00000220       ??_C@_0CD@CDGGJNPN@?$FLSSPI?3?$CFld?$FN?5NT_USER_NAME?5name?9ty@ 10005220     sspi.obj
 0002:00000244       ??_C@_0CA@JGNPMEEC@?$FLSSPI?3?$CFld?$FN?5KRB5_NAME?5name?9type?6@ 10005244     sspi.obj
 0002:00000264       ??_C@_0CL@CNJPHLHB@?$FLSSPI?3?$CFld?$FN?5NT_HOSTBASED_SERVICE@ 10005264     sspi.obj
 0002:00000290       ??_C@_0CF@KDMPIPAK@?$FLSSPI?3?$CFld?$FN?5NT_EXPORT_NAME?5name?9@ 10005290     sspi.obj
 0002:000002b8       ??_C@_0M@BOLDDFOC@UNKNOWN?5OID@ 100052b8     sspi.obj
 0002:000002c4       ??_C@_0BM@LGCLMFGL@?$FLSSPI?3?$CFld?$FN?5OID?5set?5is?5NULL?6@ 100052c4     sspi.obj
 0002:000002e0       ??_C@_0CE@OCBOPLKC@?$FLSSPI?3?$CFld?$FN?5gss_OID_set?4count?5is@ 100052e0     sspi.obj
 0002:00000304       ??_C@_1BM@OPCNFIBF@?$AAU?$AAS?$AAE?$AAR?$AAD?$AAN?$AAS?$AAD?$AAO?$AAM?$AAA?$AAI?$AAN@ 10005304     sspi.obj
 0002:00000320       ??_C@_13EFKPHINO@?$AA?$EA@ 10005320     sspi.obj
 0002:00000324       ??_C@_0CG@LCALBIAD@?$FLSSPI?3?$CFld?$FN?5get_full_name?5return@ 10005324     sspi.obj
 0002:0000034c       ??_C@_0DA@IOIDMGH@?$FLSSPI?3?$CFld?$FN?5?$DO?$DO?$DO?$DO?5Calling?5gss_rel@ 1000534c     sspi.obj
 0002:0000037c       ??_C@_0CM@BFKEACFF@?$FLSSPI?3?$CFld?$FN?5?$DO?$DO?$DO?$DO?5Calling?5gss_imp@ 1000537c     sspi.obj
 0002:000003a8       ??_C@_0CB@KBAAIDKM@?$FLSSPI?3?$CFld?$FN?5import_name?5from?5?$CFls@ 100053a8     sspi.obj
 0002:000003d0       ??_C@_1EE@BFAIICGI@?$AA?$EA?$AAW?$AAE?$AAL?$AAL?$AAK?$AAN?$AAO?$AAW?$AAN?$AA?3?$AAO?$AAR?$AAG?$AA?4@ 100053d0     sspi.obj
 0002:00000414       ??_C@_0CH@JKPPJJKG@?$FLSSPI?3?$CFld?$FN?5Host?9based?5service?5n@ 10005414     sspi.obj
 0002:0000043c       ??_C@_0BP@EGPHGJOH@?$FLSSPI?3?$CFld?$FN?5import_name?5to?5?$CFls?6@ 1000543c     sspi.obj
 0002:0000045c       ??_C@_0CN@JGBLGDBA@?$FLSSPI?3?$CFld?$FN?5?$DO?$DO?$DO?$DO?5Calling?5gss_com@ 1000545c     sspi.obj
 0002:0000048c       ??_C@_0CC@CFBGDMPH@?$FLSSPI?3?$CFld?$FN?5Comparing?5?$CFls?5and?5?$CFl@ 1000548c     sspi.obj
 0002:000004b0       ??_C@_1CM@BFAMBNFD@?$AA?$CB?$AAx?$AA?9?$AAs?$AAy?$AAs?$AA?9?$AAd?$AAe?$AAf?$AAa?$AAu?$AAl?$AAt?$AA?9@ 100054b0     sspi.obj
 0002:000004dc       ??_C@_0DC@GAAALDEK@?$FLSSPI?3?$CFld?$FN?5?$DO?$DO?$DO?$DO?5Calling?5gss_can@ 100054dc     sspi.obj
 0002:00000510       ??_C@_0DA@KPBOPIMJ@?$FLSSPI?3?$CFld?$FN?5Cannot?5canonicalize?5@ 10005510     sspi.obj
 0002:00000540       ??_C@_0CM@MFGDPAFJ@?$FLSSPI?3?$CFld?$FN?5?$DO?$DO?$DO?$DO?5Calling?5gss_exp@ 10005540     sspi.obj
 0002:0000056c       ??_C@_0CG@DOIJOALD@?$FLSSPI?3?$CFld?$FN?5Make?5fullname?3?5?$CFls?5?9@ 1000556c     sspi.obj
 0002:00000594       ??_C@_0CN@NEEPPIPL@?$FLSSPI?3?$CFld?$FN?5?$DO?$DO?$DO?$DO?5Calling?5gss_dis@ 10005594     sspi.obj
 0002:000005c4       ??_C@_0CH@MLAPIHLF@?$FLSSPI?3?$CFld?$FN?5Name?5found?3?5?$CFls?5?9?$DO?5?$CF@ 100055c4     sspi.obj
 0002:000005ec       ??_C@_0CN@MBPKOHOJ@?$FLSSPI?3?$CFld?$FN?5?$DO?$DO?$DO?$DO?5Calling?5gss_acq@ 100055ec     sspi.obj
 0002:0000061c       ??_C@_0DA@MEFNCJAE@?$FLSSPI?3?$CFld?$FN?5AcquireCredentialsHa@ 1000561c     sspi.obj
 0002:0000064c       ??_C@_0BI@FDGHJCFE@?$FLSSPI?3?$CFld?$FN?5reqKerberos?6@ 1000564c     sspi.obj
 0002:00000664       ??_C@_0BG@BIAGCKNC@?$FLSSPI?3?$CFld?$FN?5reqSPNEGO?6@ 10005664     sspi.obj
 0002:0000067c       ??_C@_1BC@KFNANHG@?$AAK?$AAe?$AAr?$AAb?$AAe?$AAr?$AAo?$AAs@ 1000567c     sspi.obj
 0002:00000690       ??_C@_1BE@ELFOBFGL@?$AAN?$AAe?$AAg?$AAo?$AAt?$AAi?$AAa?$AAt?$AAe@ 10005690     sspi.obj
 0002:000006a4       ??_C@_0BA@MCNOMCIK@cred?5expiration@ 100056a4     sspi.obj
 0002:000006b4       ??_C@_0DK@LJKKNAPH@?$FLSSPI?3?$CFld?$FN?5Acquiring?5cred?5with?5@ 100056b4     sspi.obj
 0002:000006f0       ??_C@_0DD@JHPOCMI@?$FLSSPI?3?$CFld?$FN?5Cannot?5get?5owner?5nam@ 100056f0     sspi.obj
 0002:00000724       ??_C@_0CB@MJBBLEC@?$FLSSPI?3?$CFld?$FN?5Comparing?5result?3?5?$CFd@ 10005724     sspi.obj
 0002:00000748       ??_C@_0CN@MJNIACNJ@?$FLSSPI?3?$CFld?$FN?5?$DO?$DO?$DO?$DO?5Calling?5gss_rel@ 10005748     sspi.obj
 0002:00000778       ??_C@_0CN@COKAOKCO@?$FLSSPI?3?$CFld?$FN?5?$DO?$DO?$DO?$DO?5Calling?5gss_inq@ 10005778     sspi.obj
 0002:000007a8       ??_C@_0CE@FHNLIILE@?$FLSSPI?3?$CFld?$FN?5Allocate?5new?5name?5at@ 100057a8     sspi.obj
 0002:000007d0       ??_C@_0EB@FFCALPCH@?$FLSSPI?3?$CFld?$FN?5?$DO?$DO?$DO?$DO?5Calling?5UNIMPLE@ 100057d0     sspi.obj
 0002:00000814       ??_C@_0DB@DJAAKGNJ@?$FLSSPI?3?$CFld?$FN?5?$DO?$DO?$DO?$DO?5Calling?5gss_ini@ 10005814     sspi.obj
 0002:00000848       ??_C@_0BL@BBOFLDIJ@?$FLSSPI?3?$CFld?$FN?5First?5time?$DP?5?$CFd?6@ 10005848     sspi.obj
 0002:00000864       ??_C@_0CE@FOJJGGJF@?$FLSSPI?3?$CFld?$FN?5Find?5SPNEGO?5credenti@ 10005864     sspi.obj
 0002:00000888       ??_C@_0CG@NFCFPBLP@?$FLSSPI?3?$CFld?$FN?5Find?5Kerberos?5creden@ 10005888     sspi.obj
 0002:000008b0       ??_C@_0DE@HCDAGCDE@?$FLSSPI?3?$CFld?$FN?5No?5credentials?5provi@ 100058b0     sspi.obj
 0002:000008e4       ??_C@_0CN@OKAGLDFF@?$FLSSPI?3?$CFld?$FN?5InitializeSecurityCo@ 100058e4     sspi.obj
 0002:00000918       ??_C@_0EK@GLKKIOEO@?$FLSSPI?3?$CFld?$FN?5cbMaxSignature?3?5?$CFld?4@ 10005918     sspi.obj
 0002:00000964       ??_C@_0BL@CKLNDBGC@?$FLSSPI?3?$CFld?$FN?5Names?4?5?$CFls?5?$CFls?6@ 10005964     sspi.obj
 0002:00000980       ??_C@_0EB@INHALGEB@?$FLSSPI?3?$CFld?$FN?5?$DO?$DO?$DO?$DO?5Calling?5UNIMPLE@ 10005980     sspi.obj
 0002:000009c8       ??_C@_0FD@CCKKKMJB@?$FLSSPI?3?$CFld?$FN?5gss_accept_sec_conte@ 100059c8     sspi.obj
 0002:00000a1c       ??_C@_0DA@FEKBBIAO@?$FLSSPI?3?$CFld?$FN?5?$DO?$DO?$DO?$DO?5Calling?5gss_inq@ 10005a1c     sspi.obj
 0002:00000a4c       ??_C@_0DD@CGCFJEMD@?$FLSSPI?3?$CFld?$FN?5?$DO?$DO?$DO?$DO?5Calling?5gss_del@ 10005a4c     sspi.obj
 0002:00000a80       ??_C@_0DJ@BECGEJED@?$FLSSPI?3?$CFld?$FN?5?$DO?$DO?$DO?$DO?5Calling?5IMPLEME@ 10005a80     sspi.obj
 0002:00000abc       ??_C@_0O@PNKJBMAD@context?5start@ 10005abc     sspi.obj
 0002:00000acc       ??_C@_0P@MKNAEBII@context?5expiry@ 10005acc     sspi.obj
 0002:00000adc       ??_C@_0DA@JHKOOKLJ@?$FLSSPI?3?$CFld?$FN?5?$DO?$DO?$DO?$DO?5Calling?5gss_wra@ 10005adc     sspi.obj
 0002:00000b10       ??_C@_0EB@LHLLOABD@?$FLSSPI?3?$CFld?$FN?5?$DO?$DO?$DO?$DO?5Calling?5UNIMPLE@ 10005b10     sspi.obj
 0002:00000b54       ??_C@_0CI@NNGLCOBI@?$FLSSPI?3?$CFld?$FN?5?$DO?$DO?$DO?$DO?5Calling?5gss_get@ 10005b54     sspi.obj
 0002:00000b7c       ??_C@_0CL@IAFIDLPP@?$FLSSPI?3?$CFld?$FN?5?$DO?$DO?$DO?$DO?5Calling?5gss_ver@ 10005b7c     sspi.obj
 0002:00000ba8       ??_C@_0CF@GBLMDHPG@?$FLSSPI?3?$CFld?$FN?5?$DO?$DO?$DO?$DO?5Calling?5gss_wra@ 10005ba8     sspi.obj
 0002:00000bd0       ??_C@_0CH@GBPBLBLH@?$FLSSPI?3?$CFld?$FN?5?$DO?$DO?$DO?$DO?5Calling?5gss_unw@ 10005bd0     sspi.obj
 0002:00000bf8       ??_C@_0CP@INMGJLBC@?$FLSSPI?3?$CFld?$FN?5?$DO?$DO?$DO?$DO?5Calling?5gss_ind@ 10005bf8     sspi.obj
 0002:00000c28       ??_C@_0DC@LPJJLHAH@?$FLSSPI?3?$CFld?$FN?5EnumerateSecurityPac@ 10005c28     sspi.obj
 0002:00000c5c       ??_C@_0BL@FKEDKDJG@?$FLSSPI?3?$CFld?$FN?5?$CD?$CFd?3?5?$CFls?0?5?$CFls?6?6@ 10005c5c     sspi.obj
 0002:00000c78       ??_C@_0DH@FBBCCAFO@?$FLSSPI?3?$CFld?$FN?5?$DO?$DO?$DO?$DO?5Calling?5gss_inq@ 10005c78     sspi.obj
 0002:00000cb0       ??_C@_0DD@BKGCAJOI@?$FLSSPI?3?$CFld?$FN?5?$DO?$DO?$DO?$DO?5Calling?5gss_add@ 10005cb0     sspi.obj
 0002:00000ce4       ??_C@_0CP@MAEAIKLL@?$FLSSPI?3?$CFld?$FN?5?$DO?$DO?$DO?$DO?5Calling?5gss_dis@ 10005ce4     sspi.obj
 0002:00000d14       ??_C@_09ODALAEHO@?$CI?$CFlx?$CJ?5?$CFls@ 10005d14     sspi.obj
 0002:00000d20       ??_C@_0O@HMKNBDND@status?5is?5?$CFlx@ 10005d20     sspi.obj
 0002:00000d30       ??_C@_0DF@ENDFDEMH@?$FLSSPI?3?$CFld?$FN?5?$DO?$DO?$DO?$DO?5Calling?5gss_cre@ 10005d30     sspi.obj
 0002:00000d68       ??_C@_0DA@GKLHDDIB@?$FLSSPI?3?$CFld?$FN?5?$DO?$DO?$DO?$DO?5Calling?5gss_rel@ 10005d68     sspi.obj
 0002:00000d98       ??_C@_0CP@DMCCHLKF@?$FLSSPI?3?$CFld?$FN?5?$DO?$DO?$DO?$DO?5Calling?5gss_rel@ 10005d98     sspi.obj
 0002:00000dc7       ?nothrow@std@@3Unothrow_t@1@B 10005dc7     msvcprt:nothrow.obj
 0002:00000dd0       __pDefaultRawDllMain       10005dd0     MSVCRT:dll_dllmain.obj
 0002:00000dd0       __pRawDllMain              10005dd0     MSVCRT:dll_dllmain.obj
 0002:00000dd8       ??_7exception@std@@6B@     10005dd8     MSVCRT:throw_bad_alloc.obj
 0002:00000de0       ??_C@_0BC@EOODALEL@Unknown?5exception@ 10005de0     MSVCRT:throw_bad_alloc.obj
 0002:00000df8       ??_7bad_alloc@std@@6B@     10005df8     MSVCRT:throw_bad_alloc.obj
 0002:00000e00       ??_C@_0P@GHFPNOJB@bad?5allocation@ 10005e00     MSVCRT:throw_bad_alloc.obj
 0002:00000e14       ??_7bad_array_new_length@std@@6B@ 10005e14     MSVCRT:throw_bad_alloc.obj
 0002:00000e1c       ??_C@_0BF@KINCDENJ@bad?5array?5new?5length@ 10005e1c     MSVCRT:throw_bad_alloc.obj
 0002:00000e38       ??_7type_info@@6B@         10005e38     MSVCRT:std_type_info_static.obj
 0002:00000eb0       __load_config_used         10005eb0     MSVCRT:loadcfg.obj
 0002:00000f68       ??_R4exception@std@@6B@    10005f68     MSVCRT:throw_bad_alloc.obj
 0002:00000f7c       ??_R3exception@std@@8      10005f7c     MSVCRT:throw_bad_alloc.obj
 0002:00000f8c       ??_R2exception@std@@8      10005f8c     MSVCRT:throw_bad_alloc.obj
 0002:00000f94       ??_R1A@?0A@EA@exception@std@@8 10005f94     MSVCRT:throw_bad_alloc.obj
 0002:00000fb0       ??_R4bad_alloc@std@@6B@    10005fb0     MSVCRT:throw_bad_alloc.obj
 0002:00000fc4       ??_R3bad_alloc@std@@8      10005fc4     MSVCRT:throw_bad_alloc.obj
 0002:00000fd4       ??_R2bad_alloc@std@@8      10005fd4     MSVCRT:throw_bad_alloc.obj
 0002:00000fe0       ??_R1A@?0A@EA@bad_alloc@std@@8 10005fe0     MSVCRT:throw_bad_alloc.obj
 0002:00000ffc       ??_R4bad_array_new_length@std@@6B@ 10005ffc     MSVCRT:throw_bad_alloc.obj
 0002:00001010       ??_R3bad_array_new_length@std@@8 10006010     MSVCRT:throw_bad_alloc.obj
 0002:00001020       ??_R2bad_array_new_length@std@@8 10006020     MSVCRT:throw_bad_alloc.obj
 0002:00001030       ??_R1A@?0A@EA@bad_array_new_length@std@@8 10006030     MSVCRT:throw_bad_alloc.obj
 0002:0000104c       ??_R4type_info@@6B@        1000604c     MSVCRT:std_type_info_static.obj
 0002:00001060       ??_R3type_info@@8          10006060     MSVCRT:std_type_info_static.obj
 0002:00001070       ??_R2type_info@@8          10006070     MSVCRT:std_type_info_static.obj
 0002:00001078       ??_R1A@?0A@EA@type_info@@8 10006078     MSVCRT:std_type_info_static.obj
 0002:00001094       ___safe_se_handler_table   10006094     <linker-defined>
 0002:00001380       ___rtc_iaa                 10006380     MSVCRT:initsect.obj
 0002:00001384       ___rtc_izz                 10006384     MSVCRT:initsect.obj
 0002:00001388       ___rtc_taa                 10006388     MSVCRT:initsect.obj
 0002:0000138c       ___rtc_tzz                 1000638c     MSVCRT:initsect.obj
 0002:0000146c       __TI2?AVbad_alloc@std@@    1000646c     MSVCRT:throw_bad_alloc.obj
 0002:0000147c       __CTA2?AVbad_alloc@std@@   1000647c     MSVCRT:throw_bad_alloc.obj
 0002:00001488       __CT??_R0?AVbad_alloc@std@@@8??0bad_alloc@std@@QAE@ABV01@@Z12 10006488     MSVCRT:throw_bad_alloc.obj
 0002:000014a4       __CT??_R0?AVexception@std@@@8??0exception@std@@QAE@ABV01@@Z12 100064a4     MSVCRT:throw_bad_alloc.obj
 0002:000014c0       __TI3?AVbad_array_new_length@std@@ 100064c0     MSVCRT:throw_bad_alloc.obj
 0002:000014d0       __CTA3?AVbad_array_new_length@std@@ 100064d0     MSVCRT:throw_bad_alloc.obj
 0002:000014e0       __CT??_R0?AVbad_array_new_length@std@@@8??0bad_array_new_length@std@@QAE@ABV01@@Z12 100064e0     MSVCRT:throw_bad_alloc.obj
 0002:00001860       __IMPORT_DESCRIPTOR_Secur32 10006860     secur32:Secur32.dll
 0002:00001874       __IMPORT_DESCRIPTOR_KERNEL32 10006874     kernel32:KERNEL32.dll
 0002:00001888       __IMPORT_DESCRIPTOR_VCRUNTIME140 10006888     vcruntime:VCRUNTIME140.dll
 0002:0000189c       __IMPORT_DESCRIPTOR_api-ms-win-crt-runtime-l1-1-0 1000689c     ucrt:api-ms-win-crt-runtime-l1-1-0.dll
 0002:000018b0       __IMPORT_DESCRIPTOR_api-ms-win-crt-string-l1-1-0 100068b0     ucrt:api-ms-win-crt-string-l1-1-0.dll
 0002:000018c4       __IMPORT_DESCRIPTOR_api-ms-win-crt-heap-l1-1-0 100068c4     ucrt:api-ms-win-crt-heap-l1-1-0.dll
 0002:000018d8       __IMPORT_DESCRIPTOR_api-ms-win-crt-environment-l1-1-0 100068d8     ucrt:api-ms-win-crt-environment-l1-1-0.dll
 0002:000018ec       __IMPORT_DESCRIPTOR_api-ms-win-crt-stdio-l1-1-0 100068ec     ucrt:api-ms-win-crt-stdio-l1-1-0.dll
 0002:00001900       __NULL_IMPORT_DESCRIPTOR   10006900     secur32:Secur32.dll
 0003:00000000       _KRB5_OID                  10008000     sspi.obj
 0003:00000008       _SPNEGO_OID                10008008     sspi.obj
 0003:00000010       _USER_NAME_OID             10008010     sspi.obj
 0003:00000018       _KRB5_NAME_OID             10008018     sspi.obj
 0003:00000020       _HOST_SERVICE_NAME_OID     10008020     sspi.obj
 0003:00000028       _EXPORT_NAME_OID           10008028     sspi.obj
 0003:00000030       ___security_cookie_complement 10008030     MSVCRT:gs_cookie.obj
 0003:00000034       ___security_cookie         10008034     MSVCRT:gs_cookie.obj
 0003:00000038       ___scrt_native_dllmain_reason 10008038     MSVCRT:utility.obj
 0003:00000040       ___isa_enabled             10008040     MSVCRT:cpu_disp.obj
 0003:00000044       ___scrt_ucrt_dll_is_in_use 10008044     MSVCRT:ucrt_stubs.obj
 0003:00000048       ??_R0?AVbad_alloc@std@@@8  10008048     MSVCRT:throw_bad_alloc.obj
 0003:00000064       ??_R0?AVexception@std@@@8  10008064     MSVCRT:throw_bad_alloc.obj
 0003:00000080       ??_R0?AVbad_array_new_length@std@@@8 10008080     MSVCRT:throw_bad_alloc.obj
 0003:000000a8       ??_R0?AVtype_info@@@8      100080a8     MSVCRT:std_type_info_static.obj
 0003:000000c0       ?_OptionsStorage@?1??__local_stdio_printf_options@@9@4_KA 100080c0     sspi.obj
 0003:000000c8       _trace                     100080c8     sspi.obj
 0003:000003f0       ?__type_info_root_node@@3U__type_info_node@@A 100083f0     MSVCRT:tncleanup.obj
 0003:000003f8       ?_OptionsStorage@?1??__local_stdio_scanf_options@@9@4_KA 100083f8     MSVCRT:default_local_stdio_options.obj
 0003:00000400       ___scrt_current_native_startup_state 10008400     MSVCRT:utility.obj
 0003:00000404       ___scrt_native_startup_lock 10008404     MSVCRT:utility.obj
 0003:00000424       ___scrt_debugger_hook_flag 10008424     MSVCRT:utility_desktop.obj
 0003:00000428       ___isa_available           10008428     MSVCRT:cpu_disp.obj
 0003:0000042c       ___favor                   1000842c     MSVCRT:cpu_disp.obj
 0003:00000430       ___dyn_tls_init_callback   10008430     <common>

 entry point at        0001:0000308a

 Static symbols

 0000:ffff5000       .debug$S                   10000000     sspi_bridge.exp
 0000:ffff5000       .debug$S                   10000000     vcruntime:VCRUNTIME140.dll
 0000:ffff5000       .debug$S                   10000000     vcruntime:VCRUNTIME140.dll
 0000:ffff5000       .debug$S                   10000000     vcruntime:VCRUNTIME140.dll
 0000:ffff5000       .debug$S                   10000000     vcruntime:VCRUNTIME140.dll
 0000:ffff5000       .debug$S                   10000000     vcruntime:VCRUNTIME140.dll
 0000:ffff5000       .debug$S                   10000000     vcruntime:VCRUNTIME140.dll
 0000:ffff5000       .debug$S                   10000000     vcruntime:VCRUNTIME140.dll
 0000:ffff5000       .debug$S                   10000000     vcruntime:VCRUNTIME140.dll
 0000:ffff5000       .debug$S                   10000000     vcruntime:VCRUNTIME140.dll
 0000:ffff5000       .debug$S                   10000000     vcruntime:VCRUNTIME140.dll
 0000:ffff5000       .debug$S                   10000000     vcruntime:VCRUNTIME140.dll
 0000:ffff5000       .debug$S                   10000000     ucrt:api-ms-win-crt-environment-l1-1-0.dll
 0000:ffff5000       .debug$S                   10000000     ucrt:api-ms-win-crt-environment-l1-1-0.dll
 0000:ffff5000       .debug$S                   10000000     ucrt:api-ms-win-crt-heap-l1-1-0.dll
 0000:ffff5000       .debug$S                   10000000     ucrt:api-ms-win-crt-heap-l1-1-0.dll
 0000:ffff5000       .debug$S                   10000000     ucrt:api-ms-win-crt-heap-l1-1-0.dll
 0000:ffff5000       .debug$S                   10000000     ucrt:api-ms-win-crt-runtime-l1-1-0.dll
 0000:ffff5000       .debug$S                   10000000     ucrt:api-ms-win-crt-runtime-l1-1-0.dll
 0000:ffff5000       .debug$S                   10000000     ucrt:api-ms-win-crt-runtime-l1-1-0.dll
 0000:ffff5000       .debug$S                   10000000     ucrt:api-ms-win-crt-runtime-l1-1-0.dll
 0000:ffff5000       .debug$S                   10000000     ucrt:api-ms-win-crt-runtime-l1-1-0.dll
 0000:ffff5000       .debug$S                   10000000     ucrt:api-ms-win-crt-runtime-l1-1-0.dll
 0000:ffff5000       .debug$S                   10000000     ucrt:api-ms-win-crt-runtime-l1-1-0.dll
 0000:ffff5000       .debug$S                   10000000     ucrt:api-ms-win-crt-runtime-l1-1-0.dll
 0000:ffff5000       .debug$S                   10000000     ucrt:api-ms-win-crt-runtime-l1-1-0.dll
 0000:ffff5000       .debug$S                   10000000     ucrt:api-ms-win-crt-runtime-l1-1-0.dll
 0000:ffff5000       .debug$S                   10000000     ucrt:api-ms-win-crt-runtime-l1-1-0.dll
 0000:ffff5000       .debug$S                   10000000     ucrt:api-ms-win-crt-runtime-l1-1-0.dll
 0000:ffff5000       .debug$S                   10000000     ucrt:api-ms-win-crt-runtime-l1-1-0.dll
 0000:ffff5000       .debug$S                   10000000     ucrt:api-ms-win-crt-runtime-l1-1-0.dll
 0000:ffff5000       .debug$S                   10000000     ucrt:api-ms-win-crt-stdio-l1-1-0.dll
 0000:ffff5000       .debug$S                   10000000     ucrt:api-ms-win-crt-stdio-l1-1-0.dll
 0000:ffff5000       .debug$S                   10000000     ucrt:api-ms-win-crt-stdio-l1-1-0.dll
 0000:ffff5000       .debug$S                   10000000     ucrt:api-ms-win-crt-stdio-l1-1-0.dll
 0000:ffff5000       .debug$S                   10000000     ucrt:api-ms-win-crt-string-l1-1-0.dll
 0000:ffff5000       .debug$S                   10000000     ucrt:api-ms-win-crt-string-l1-1-0.dll
 0000:ffff5000       .debug$S                   10000000     ucrt:api-ms-win-crt-string-l1-1-0.dll
 0000:ffff5000       .debug$S                   10000000     ucrt:api-ms-win-crt-string-l1-1-0.dll
 0000:ffff5000       .debug$S                   10000000     ucrt:api-ms-win-crt-string-l1-1-0.dll
 0000:ffff5000       .debug$S                   10000000     kernel32:KERNEL32.dll
 0000:ffff5000       .debug$S                   10000000     kernel32:KERNEL32.dll
 0000:ffff5000       .debug$S                   10000000     kernel32:KERNEL32.dll
 0000:ffff5000       .debug$S                   10000000     kernel32:KERNEL32.dll
 0000:ffff5000       .debug$S                   10000000     kernel32:KERNEL32.dll
 0000:ffff5000       .debug$S                   10000000     kernel32:KERNEL32.dll
 0000:ffff5000       .debug$S                   10000000     kernel32:KERNEL32.dll
 0000:ffff5000       .debug$S                   10000000     kernel32:KERNEL32.dll
 0000:ffff5000       .debug$S                   10000000     kernel32:KERNEL32.dll
 0000:ffff5000       .debug$S                   10000000     kernel32:KERNEL32.dll
 0000:ffff5000       .debug$S                   10000000     kernel32:KERNEL32.dll
 0000:ffff5000       .debug$S                   10000000     kernel32:KERNEL32.dll
 0000:ffff5000       .debug$S                   10000000     kernel32:KERNEL32.dll
 0000:ffff5000       .debug$S                   10000000     kernel32:KERNEL32.dll
 0000:ffff5000       .debug$S                   10000000     kernel32:KERNEL32.dll
 0000:ffff5000       .debug$S                   10000000     kernel32:KERNEL32.dll
 0000:ffff5000       .debug$S                   10000000     kernel32:KERNEL32.dll
 0000:ffff5000       .debug$S                   10000000     kernel32:KERNEL32.dll
 0000:ffff5000       .debug$S                   10000000     kernel32:KERNEL32.dll
 0000:ffff5000       .debug$S                   10000000     kernel32:KERNEL32.dll
 0000:ffff5000       .debug$S                   10000000     kernel32:KERNEL32.dll
 0000:ffff5000       .debug$S                   10000000     secur32:Secur32.dll
 0000:ffff5000       .debug$S                   10000000     secur32:Secur32.dll
 0000:ffff5000       .debug$S                   10000000     secur32:Secur32.dll
 0000:ffff5000       .debug$S                   10000000     secur32:Secur32.dll
 0000:ffff5000       .debug$S                   10000000     secur32:Secur32.dll
 0000:ffff5000       .debug$S                   10000000     secur32:Secur32.dll
 0000:ffff5000       .debug$S                   10000000     secur32:Secur32.dll
 0000:ffff5000       .debug$S                   10000000     secur32:Secur32.dll
 0000:ffff5000       .debug$S                   10000000     secur32:Secur32.dll
 0000:ffff5000       .debug$S                   10000000     secur32:Secur32.dll
 0000:ffff5000       .debug$S                   10000000     secur32:Secur32.dll
 0000:ffff5000       .debug$S                   10000000     secur32:Secur32.dll
 0001:00000000       ??__Etrace@@YAXXZ          10001000 f   sspi.obj
 0001:0000016c       _flag_gss_to_sspi          1000116c f   sspi.obj
 0001:000001b6       _flag_sspi_to_gss          100011b6 f   sspi.obj
 0001:00000218       _get_full_name             10001218 f   sspi.obj
 0001:00002616       _has_oid                   10003616 f   sspi.obj
 0001:00002646       _is_same_oid               10003646 f   sspi.obj
 0001:00002675       _memcpy_s                  10003675 f   sspi.obj
 0001:000026f9       _new_context               100036f9 f   sspi.obj
 0001:00002737       _seconds_until             10003737 f   sspi.obj
 0001:000027a5       _show_oid                  100037a5 f   sspi.obj
 0001:000028e4       _show_oid_set              100038e4 f   sspi.obj
 0001:00002962       _show_time                 10003962 f   sspi.obj
 0001:00002c67       __catch$??2@YAPAXIABUnothrow_t@std@@@Z$0 10003c67 f   MSVCRT:new_scalar_nothrow.obj
 0001:00002ca0       $$000000                   10003ca0     MSVCRT:lldiv.obj
 0001:00002d4a       ?dllmain_crt_dispatch@@YGHQAUHINSTANCE__@@KQAX@Z 10003d4a f   MSVCRT:dll_dllmain.obj
 0001:00002d9d       ?dllmain_crt_process_attach@@YAHQAUHINSTANCE__@@QAX@Z 10003d9d f   MSVCRT:dll_dllmain.obj
 0001:00002ea4       ?dllmain_crt_process_detach@@YAH_N@Z 10003ea4 f   MSVCRT:dll_dllmain.obj
 0001:00002f54       ?dllmain_dispatch@@YAHQAUHINSTANCE__@@KQAX@Z 10003f54 f   MSVCRT:dll_dllmain.obj
 0001:0000305f       ?dllmain_raw@@YGHQAUHINSTANCE__@@KQAX@Z 1000405f f   MSVCRT:dll_dllmain.obj
 0001:000030e2       ___get_entropy             100040e2 f   MSVCRT:gs_support.obj
 0001:000031d7       ?find_pe_section@@YAPAU_IMAGE_SECTION_HEADER@@QAEI@Z 100041d7 f   MSVCRT:utility.obj
 0001:00003630       $$000000                   10004630     MSVCRT:sehprolg4.obj
 0001:00003ad0       __ehhandler$??2@YAPAXIABUnothrow_t@std@@@Z 10004ad0 f   MSVCRT:new_scalar_nothrow.obj
 0002:00000128       ?trace$initializer$@@3P6AXXZA 10005128     sspi.obj
 0002:00000dc8       _GS_ExceptionPointers      10005dc8     MSVCRT:gs_report.obj
 0002:00001390       __catchsym$??2@YAPAXIABUnothrow_t@std@@@Z$2 10006390     MSVCRT:new_scalar_nothrow.obj
 0002:000013a0       __unwindtable$??2@YAPAXIABUnothrow_t@std@@@Z 100063a0     MSVCRT:new_scalar_nothrow.obj
 0002:000013b0       __tryblocktable$??2@YAPAXIABUnothrow_t@std@@@Z 100063b0     MSVCRT:new_scalar_nothrow.obj
 0002:000013c4       __ehfuncinfo$??2@YAPAXIABUnothrow_t@std@@@Z 100063c4     MSVCRT:new_scalar_nothrow.obj
 0002:000013e8       __sehtable$?dllmain_crt_process_attach@@YAHQAUHINSTANCE__@@QAX@Z 100063e8     MSVCRT:dll_dllmain.obj
 0002:00001408       __sehtable$?dllmain_crt_process_detach@@YAH_N@Z 10006408     MSVCRT:dll_dllmain.obj
 0002:00001430       __sehtable$?dllmain_dispatch@@YAHQAUHINSTANCE__@@KQAX@Z 10006430     MSVCRT:dll_dllmain.obj
 0002:00001450       __sehtable$___scrt_is_nonwritable_in_current_image 10006450     MSVCRT:utility.obj
 0002:00001500       .edata                     10006500     sspi_bridge.exp
 0002:00001528       rgpv                       10006528     sspi_bridge.exp
 0002:00001598       rgszName                   10006598     sspi_bridge.exp
 0002:00001608       rgwOrd                     10006608     sspi_bridge.exp
 0002:00001640       szName                     10006640     sspi_bridge.exp
 0002:00001650       $N00001                    10006650     sspi_bridge.exp
 0002:00001667       $N00002                    10006667     sspi_bridge.exp
 0002:00001678       $N00003                    10006678     sspi_bridge.exp
 0002:0000168f       $N00004                    1000668f     sspi_bridge.exp
 0002:000016a5       $N00005                    100066a5     sspi_bridge.exp
 0002:000016b6       $N00006                    100066b6     sspi_bridge.exp
 0002:000016c7       $N00007                    100066c7     sspi_bridge.exp
 0002:000016e0       $N00008                    100066e0     sspi_bridge.exp
 0002:000016f7       $N00009                    100066f7     sspi_bridge.exp
 0002:00001708       $N00010                    10006708     sspi_bridge.exp
 0002:0000171b       $N00011                    1000671b     sspi_bridge.exp
 0002:0000172b       $N00012                    1000672b     sspi_bridge.exp
 0002:00001742       $N00013                    10006742     sspi_bridge.exp
 0002:0000174e       $N00014                    1000674e     sspi_bridge.exp
 0002:0000175e       $N00015                    1000675e     sspi_bridge.exp
 0002:00001775       $N00016                    10006775     sspi_bridge.exp
 0002:00001788       $N00017                    10006788     sspi_bridge.exp
 0002:0000179d       $N00018                    1000679d     sspi_bridge.exp
 0002:000017b1       $N00019                    100067b1     sspi_bridge.exp
 0002:000017c2       $N00020                    100067c2     sspi_bridge.exp
 0002:000017dd       $N00021                    100067dd     sspi_bridge.exp
 0002:000017f0       $N00022                    100067f0     sspi_bridge.exp
 0002:00001801       $N00023                    10006801     sspi_bridge.exp
 0002:00001812       $N00024                    10006812     sspi_bridge.exp
 0002:00001826       $N00025                    10006826     sspi_bridge.exp
 0002:00001831       $N00026                    10006831     sspi_bridge.exp
 0002:00001840       $N00027                    10006840     sspi_bridge.exp
 0002:00001849       $N00028                    10006849     sspi_bridge.exp
 0002:00001b4e       .idata$6                   10006b4e     secur32:Secur32.dll
 0002:00001d0c       .idata$6                   10006d0c     kernel32:KERNEL32.dll
 0002:00001dd0       .idata$6                   10006dd0     vcruntime:VCRUNTIME140.dll
 0002:00001f6a       .idata$6                   10006f6a     ucrt:api-ms-win-crt-runtime-l1-1-0.dll
 0002:00001f8c       .idata$6                   10006f8c     ucrt:api-ms-win-crt-string-l1-1-0.dll
 0002:00001fae       .idata$6                   10006fae     ucrt:api-ms-win-crt-heap-l1-1-0.dll
 0002:00001fce       .idata$6                   10006fce     ucrt:api-ms-win-crt-environment-l1-1-0.dll
 0002:00001ff4       .idata$6                   10006ff4     ucrt:api-ms-win-crt-stdio-l1-1-0.dll
 0003:000000d0       _GS_ExceptionRecord        100080d0     MSVCRT:gs_report.obj
 0003:00000120       _GS_ContextRecord          10008120     MSVCRT:gs_report.obj
 0003:000003ec       ?__proc_attached@@3HA      100083ec     MSVCRT:dll_dllmain.obj
 0003:00000408       ?is_initialized_as_dll@@3_NA 10008408     MSVCRT:utility.obj
 0003:00000409       ?module_local_atexit_table_initialized@@3_NA 10008409     MSVCRT:utility.obj
 0003:0000040c       ?module_local_atexit_table@@3U_onexit_table_t@@A 1000840c     MSVCRT:utility.obj
 0003:00000418       ?module_local_at_quick_exit_table@@3U_onexit_table_t@@A 10008418     MSVCRT:utility.obj
 0004:00000060       $R000000                   10009060     sspi_bridge.dll.res
